:030000000219FDE5
:03000B000200A848
:03002B0002015D72
:03005B000202DCC2
:030073000202C2C4
:1000800002030406080C10182030406080040608A3
:100090000C10182030406080A0C000070F1F3F05E3
:1000A000050D050205030302C2AFC0D0C0E0206207
:1000B00017E5256002E473E525F4F58A758B00D217
:1000C00062D0E0D0D0D2AF3285268AC262E526F473
:1000D000602F758B00D0E0D0D0C294C292C290D273
:1000E000AF32C294C292C290206E0C206609740591
:1000F000D5E0FDE57E4290758B00D0E0D0D0D2AF48
:1001000032758A00C28DD26201F701B730680520CE
:100110006602D29401B7306805206602D29201B718
:10012000306805206602D29001B7C29530680A2077
:1001300066077428D5E0FDD29401B7C29330680AEF
:100140002066077428D5E0FDD29201B7C2913068CD
:100150000A2066077428D5E0FDD29001B7C2AFC26D
:10016000AD53E6EFC0D0C0E0D2D3D2AFC2CEE52AC5
:100170006007207449152A21BE7800790020742E6A
:10018000E580307E01F430E40278FF53DACF207E40
:100190000343DA20307E0343DA10C2D8C271E5800F
:1001A000307E01F430E40279FFC3E89970CB30610E
:1001B00003752A18207403752A18885FD27020747A
:1001C0000DE52B6004152B21CE43DA01C2D8207037
:1001D000024130A85F206102C270207431C3E894EC
:1001E000F0400374F0F8E8C4540F28F87984B7039A
:1001F00002410EC313C3138721200802C313200A30
:1002000006C3C898F8410E28F8500374FFF8C3E8F5
:1002100095685003E568F88822E52D54066011E5DD
:1002200033C313C31324062522F52250037522FF7E
:10023000852224A824C3E52495644002A864882567
:10024000E56970024174C3E8AA699A5003E8FAE4C8
:10025000F9EAC333FBE56BF45B29400D256AF8E549
:100260006A6002156A400B41740AC3E56A9A50023B
:10027000056A78FF8826C3E52594404002D26420B1
:10028000CF0AD0E0D0D043E610D2AD32C2CF053A8B
:100290007801E52A6005307402152AC3E55F9401F0
:1002A000400575620041B8756300756C00E5622415
:1002B00001F56250037562FFD0E0D0D043E610D262
:1002C000AD32C2AFC0D053E67FC260759100855693
:1002D00094855795759104D0D0D2AF32C2AF53E612
:1002E000EFC2ADC0D0C0E0C0F0D2D3D2AFA8FBA95E
:1002F000FCC2D8307102614353DACF207E0343DA67
:1003000010307E0343DA20D271E580307E01F42084
:10031000E402611A88278928A16A53DACF207E0374
:1003200043DA20307E0343DA10C2D8C2713074023F
:10033000A1567800E580307E01F430E402A15688B1
:100340005FA13E53DACF207E0343DA20307E0343A1
:10035000DA10C271206102811C53DACF207E034380
:10036000DA10307E0343DA20C2D8D271885A895B12
:10037000C3E89558F8E99559F97B007E087A00C3DF
:10038000E8948CE994005005755E00810E88217810
:10039000A2E6A8216055C3E894C8E994005008E497
:1003A000D2E4FB7A0A61E9C3E89468E99401500851
:1003B000E4D2E3FB7A0F61E9C3E894D0E9940250F8
:1003C00008E4D2E2FB7A1E61E9C3E894A0E994054F
:1003D0005008E4D2E1FB7A3C61E9C3E89498E994DF
:1003E000085008E4D2E0FB7A787E00C3E8955CFC14
:1003F000E9955DFD30E70AECF42401FCEDF43400EE
:10040000FD755E00C3EC9AED9E5003755E01885C3D
:10041000895D855A58855B597802A13EC3E89527C6
:10042000F8E99528F9307C02A122307B02A1223024
:100430007A02A11B207502813FE9FDE8FC815EE99B
:10044000C313F9E813F8307902A11BE9C313F9E8E3
:1004500013F8307802A11BE9C313FDE813FC2061F7
:1004600026C3EC941CED940240028175ED7018C314
:0E047000EC94C850120529C3E529940A5002E5
:10047E00A156755F00D270A156E529600215297844
:10048E0088E6F97400207F087896B90302789EE614
:10049E0024FAFEE43400FFC3EC9EFCED9FFD9208AF
:1004AE00B90310A2085007207609D27681C13076A2
:1004BE0002C276A2085016B9030DECF42401FCED2D
:1004CE00F43400FD0204DB78007900A122B9031593
:1004DE00EC33FCED33FDC3EC940AFCED9400FD50BF
:1004EE00047C007D00C3EC94FFED9400400678FF81
:1004FE007900A122EC8575F0A4C5F0A2F733F87946
:10050E0000400302053E78FF790002053EE9C31361
:10051E00F9E813F8307C0EE9600278FFC3E813386F
:10052E00F8E43400F9C3E894FFE99400400278FF40
:10053E00885FD270206102A156741FF4552F4BF5BF
:10054E002FC274EB7002D274752A18307403752A98
:10055E000A306102A16A20740353DAFE2074037517
:10056E002B06D0F0D0E0D0D0D2AD43E610327901D8
:10057E0002059A790302059A790A02059A791E02F2
:10058E00059A796402059A79C802059A7817E4D516
:10059E00E0FDD8FAD9F6227A147B780205C17A10DA
:1005AE007B8C0205C17A0D7BB40205C17A0B7BC828
:1005BE000205C17902B27DE4C293D5E0FDD292D597
:1005CE00E0FDC292D5E0FDD293D5E0FDD294E57662
:1005DE00D5E0FDC2947496D5E0FDD9D9EAF8D5E000
:1005EE00FDD8FBDBCEC29322C37C007D0075F000EC
:1005FE0005F0EA33FAEB33FB50F6EB13FBEA13FA92
:10060E00C3E9FFE8FEE89AF8E99BF95004EFF9EE2A
:10061E00F8B3EC33FCED33FDD5F0DFEDF9ECF82259
:10062E00E889F08A20D2D4F8A9F07B0030F70B7B52
:10063E00FFF42401F8E9F43400F9E88520F0A4ADC4
:10064E00F0F8E98520F0A4AFF0FEED2EF974003F2E
:10065E00FA7C04C3EA13FAE913F9E813F8DCF48B15
:10066E00F030F70AE8F42401F8E9F43400F9E889E7
:10067E00F0C2D4F8A9F02222C3E54113F9E54013E4
:10068E00F8C3E54598F8E54699F9500CC3E894800F
:10069E00E994FF40160206BDC3E8947FE99400502A
:1006AE00030206BD787F79000206BD788079FF8847
:1006BE004A894B22E54A2547F8E54B3548F9854BE3
:1006CE0020E4300701F43549FA30E709C3EA94F023
:1006DE0040150206FBC3EA940F50030206FB78FF97
:1006EE0079FF7A0F0206FB780079007AF0C3E524D1
:1006FE009564500AC374019524500B020719E54BFB
:10070E0020E70E020719E54B30E706884789488A2D
:10071E00492278A4E6FAC3E54A33F8E54B33F9D11A
:10072E002EE930E70BC3E89480E994FF4013E153C0
:10073E00C3E8947FE994005002E153787F7900E199
:10074E0053788079FFE820E715C3E52398F8400930
:10075E00C3E89401400302077A780102077AE8F4AD
:10076E0024012523F8400302077A78FF884C22786B
:10077E00A5E6FAA848A949D12EE930E70CC3E894BA
:10078E0001E994FF40160207AEC3E894FFE9940016
:10079E0050030207AE78FF79000207AE780179FFA9
:1007AE00E920E715C3E54C98F84009C3E8940140E9
:1007BE00030207D578010207D5E8F42401254CF889
:1007CE0040030207D578FF88242278FFC26420698F
:1007DE003D206A12D264C3E541940A4009C3E5255F
:1007EE0094405002C26479A1E76023E541601F7412
:1007FE00FF8541F0848539F0306A0375F005A4F861
:10080E00C5F0600278FFC3E895675002A867886656
:10081E0022C3E5409440E5419401E566500314017E
:10082E0030046002F566220208382275E8902278BC
:10083E0083E6FFE5E820ECF7A8BDA9BE0573C3E586
:10084E007394084052757300E9FA79A0E76044EAA0
:10085E007007E574601B020873C3E895746010E5B9
:0F086E00745006600C1402087F0460F902087FC2
:10087D00E574F574C3946D401B7564C0C394044056
:10088D0013756480C39404400B756440C394044095
:10089D000375640075BB0E22E564F460020564E522
:1008AD0073B4070375BB1022743279A687F0A4C503
:1008BD00F0A2F733F8C3E895644002A86488228853
:1008CD0024882588268867227540007541F022C24C
:1008DD00AF75C820A8CCA9CDAA3A30CF010A75C8EA
:1008ED0024D2AFAB3BAC3C883B893CC3E89BF8E9D9
:1008FD009C206908F930670221F1214EAD3D8A3DFA
:10090D00F9EA9DFA600478FF79FFAE3EAF3F8B3E6A
:10091D008C3FC3EC9FFCC3E99CF542A83BA93CC3AB
:10092D00E89EF8E99FF9C3E54113FBE54013FAE8AA
:10093D002AF540E93BF54150067540FF7541FF2111
:10094D0098AA40AB41AC40AD417E047F02C3EB940D
:10095D000440021E1FC3EB940840021E1FC3ED137B
:10096D00FDEC13FCDEF7C3EA9CFAEB9DFBEF60098F
:10097D00C3E913F9E813F8DFF7EA28FAEB39FB8A34
:10098D00408B4150067BFF8B408B41C3EB94025053
:10099D0002D2673069047F0321C37892E6FFC3E575
:1009AD0037948240110FC3E53794A040010FC3EF78
:1009BD00940640027F057E07E541C4540FF9E541D9
:1009CD00C454F0F8E540C4540F28F8C3E89EFAE982
:1009DD009400FB4009C3EA9402EB940050047A02A0
:1009ED00E4FB413DAA40AB41EBC4FEEAC4540F4EBB
:1009FD00FCC3EA9CFAEB9400FBC3E813C313F8EABB
:100A0D0028FAEB3400FB8A408B41C3EB9402400281
:100A1D00C2677807EBC4FE7B00EAC4540F4EFAC3DD
:100A2D00EA98FA4005C3940250027A027892E6FFE2
:100A3D00306002413D855256855357D26043E68062
:100A4D00C3E49AF8E49BF930670241D7E8FAE9FB71
:100A5D00D3E913FDE813FC88528953C3EF94036067
:100A6D0038EF20E00DE82CF8E93DF9ECFAEDFB024A
:100A7D000A92E828F8E939F9C3E82402F8E93400C4
:100A8D00F97AFE7BFFC3EF9403400E8A548B558891
:100A9D004E894F8C508D51610B885489558A4E8BE0
:100AAD004F8C508D51306920C3E53394034019E5C7
:100ABD0042A2E713F8E555F4240138400B20E7086E
:100ACD007554FFF42401F555610BE8FAD3E813FCD6
:100ADD008852C3EF94036020EF20E007E82CF8EC78
:100AED00FA41F7E8282402F87AFEC3EF9403400890
:100AFD008A54884E8C50610B88548A4E8C50E56B0D
:100B0D00C3335002646BF56B3060026115753402AE
:100B1D00D26043E680E52D54066026A840A941C366
:100B2D00E913F9E813F8C2AF53E67F759100C3E4FA
:100B3D0098F594E499F595759104D26043E680D2C9
:100B4D00AF22D265754400752000306B03752040CF
:100B5D00020B6ED265754400752040306B03752015
:100B6D0000D2AF7801206722E52D54066002C265E0
:100B7D00C3E5419405401378029405400878039429
:100B8D000540027806306902780A206019E5446054
:100B9D001530690AC3E53394034003D53406D2AF4B
:100BAD00D26C8140711DD2AF0000C2AF206726E527
:100BBD0041C3FB940F40027B0FEB240530730123DF
:100BCD00306A02742820620123F93069027982E5C6
:100BDD008BC39940B50544E59BF45440B520028183
:100BED002A30690A08C3E8940A4001086197206514
:100BFD0002616EC26553E67F759100306710759482
:100C0D00007595FE759104D26043E680616EAE402D
:100C1D00AF41C3E49EF594E49FF5958111C3E5338F
:100C2D0094025002616E306502616ED802813E61A0
:100C3D0097C26C53E67F75910085549485559575D3
:100C4D009104854E56854F57D26043E680D2AFE56D
:100C5D002D54066008206A020533020C7A306C0DA3
:0E0C6D00206B0A206507158115810214F12203
:100C7B0078003064053065027801E53775F007A41C
:100C8B00F9E5F028F5F0E9A2F013A2F113A2F213A3
:100C9B00F537C394785003753778C3E537953840EB
:100CAB0008D266C294C292C29030600281B4855061
:100CBB0056855157D26043E68022207D11C2AF7515
:100CCB004302C293D295D2AF759F70020E94C2AFFE
:100CDB00754302C293D291D2AF759F70020E9430BE
:100CEB007243207D20C2AF75430390013B757E0894
:100CFB00C290C291306204D292A108D293D2AF7546
:100D0B009F00020E94C2AF75430390013B757E08A2
:100D1B00C294C295306204D292A128D293D2AF75FD
:100D2B009F20020E94207D17C2AF754303900116CE
:100D3B00C290306202D292D2AF759F00020E94C263
:100D4B00AF754303900116C294306202D292D2AFB8
:100D5B00759F20020E94207D11C2AF754304C2957E
:100D6B00D291D2AF759F20020E94C2AF754304C2CD
:100D7B0091D295D2AF759F00020E94307243207DB5
:100D8B0020C2AF75430590012A757E20C292C29393
:100D9B00306204D294A1A4D295D2AF759F70020E8B
:100DAB0094C2AF75430590014C757E02C292C293FB
:100DBB00306204D290A1C4D291D2AF759F70020E53
:100DCB0094207D17C2AF75430590010CC29230621F
:100DDB0002D294D2AF759F70020E94C2AF754305C9
:100DEB00900120C2923062EBD290D2AF759F70020D
:100DFB000E94207D11C2AF754306C291D293D2AF30
:100E0B00759F00020E94C2AF754306C295D293D262
:100E1B00AF759F20020E94307242207D20C2AF75B9
:100E2B00430190014C757E02C294C295306204D28C
:100E3B0090C140D291D2AF759F20020E94C2AF7574
:100E4B00430190012A757E20C290C291306204D278
:100E5B0094C160D295D2AF759F00C194207D16C20C
:100E6B00AF754301900120C294306202D290D2AF91
:100E7B00759F20C194C2AF75430190010CC2903095
:100E8B006202D294D2AF759F00C2662290010A759E
:100E9B007E00C294C292C290C295C293C291C262AA
:100EAB0022788076FF0876FF0876FF0876FF0876B3
:100EBB000308760408760A0876010876010876019D
:100ECB00788C76010876FF0876FF0876FF0876FFA8
:100EDB000876FF0876030876FF0876FF0876FF088A
:100EEB0076250876D00876FA0876FA08760408761E
:100EFB00FF08760108760008767A0876FF087601F7
:100F0B00087601087600087603227887E6FFC2721E
:100F1B007888E6C394036008C27DE630E102D27D97
:100F2B00C27E7889E630E102D27EC3EF940260087C
:100F3B00758E01D273020F48758E00C273227880B2
:100F4B00E6149000809378A4F67881E614900080E4
:100F5B009378A5F67886E61490008D9378A6F678AC
:100F6B009CE67538FF75390CB402067538A07539D7
:100F7B000AB4030675388275390578A3E614900018
:100F8B009A93F569D19722227896E6FA7897E6FB41
:100F9B007888E6B40305C3EB940EFB307F047A002C
:100FAB007BFFC3EB9AFCC3948250027C8275750065
:100FBB000575EC8575F0A4C3E5F0947D40F222D263
:100FCB007FF19312058B7A007B007C10120581E573
:100FDB005F2AFA74003BFBDCF37C04C3EB13FBEAE4
:100FEB0013FADCF7FEC27FF19322E5EF20E60375DF
:100FFB0020000520903FFFE520146006901DFF1494
:10100B0060009304600375EF1253D9BF7581C04321
:10101B00FF8012057C75EF0243B203E5B324042075
:10102B00E70DF521E5E320E0068521B343E301124B
:10103B000E977580FF75A40075F1DC75D4EF759074
:10104B00C075A53F75F23F75D5C075A60175E24118
:10105B00E4F8F6D8FD756B01120EAC1215337898C7
:0D106B008676753001C2AF1205951205A5FD
:1010780012058B1205AC12058B1205B312058B12E3
:10108800164C120595120595120590C2AF78FA799B
:10109800FA308407D9FBD8F7021C00120F15120F7B
:1010A80049120F92120F9378988676120E977588C8
:1010B8005075891275C82475910475D84075A82291
:1010C80075B80275E690759B80759D0075D10E7593
:1010D800BC5875BB0E75BA1175E88012057CD2AF85
:1010E80012083553DACF207E0343DA20307E0343DB
:1010F800DA1043DA01C2D8C271120595D2617B03B6
:101108007A0CE55E70077A0CDB0302109312058BEC
:10111800207003021093C270E55FC3940240E1E5BA
:101128002F541F856160F561B560D5DAD5C261536A
:10113800DACF207E0343DA20307E0343DA10C2D8A8
:10114800C27178A2E67008D274E52F54E0F52FC278
:1011580075752900120590307409C3E529940A4071
:1011680002D27512058178023074027800C3E55FF7
:101178009840F0C2AF1205A51205A51205A5D2AF79
:10118800120595754D007888E6B40302417312057F
:1011980081788CE6C394015003021273E530C3943E
:1011A800015003021273207435C3E55F94FF5003A6
:1011B800021273C2AF1205BAD2AF120590C3E55F2F
:1011C800940150EFC2AF1205A51205861205A5D2EB
:1011D800AF120590C3E55F94FF40E90216D17F0581
:1011E800D27F120F93120590C2AFC27F120F93AE37
:1011F8005FC3E55F947FD2AF407B12057CC2AF121C
:1012080005BAD2AFDFDA120FCAC3EE94057897F6A3
:101218001205951215751216547F0AD27F120F9374
:10122800120590C2AFC27F120F93AE5FC3E55F9401
:101238007FD2AF50E412057CC2AF1205A512058615
:101248001205A5D2AFDFD4120FCAEE24057896F6A0
:10125800120595121575121683120590120F93C375
:10126800E55F94FF500221AE0216D1C3E55F954DAC
:101278004003855F4D12059078017988E7B4030231
:101288007805C3E55F984002218EC2AF1205BA12F5
:1012980005BA1205BAD2AF120595753000E4F531DA
:1012A800F5320531E531F470390532789AE6781966
:1012B800146012783214600D787D14600878FA147E
:1012C8006003753200C3E53298401715327531B4A2
:1012D80078998676C2AF1205BAD2AF789886761218
:1012E8000590120586E52A7005307402019378018D
:1012F8002074027806C3E55F9840A77888E6C3940F
:10130800036003120590E52A7003021093C2AF121E
:101318000E97E4F522F523F524F525F526F56AD28E
:10132800AF7885E6C333F568E4F545F546F547F546
:1013380048F549F573F52CF52DF53775730875BB28
:101348001012057C120839E5E820ECFBA8BDA9BEFF
:10135800E97001F8887412083D75730875BB107838
:1013680087E6FE7602120F157887EEF6C2AF75642F
:10137800FF1208B5852264852265852266D2AF757D
:10138800220175240175250175260185636C756D2B
:10139800017888E6B40307C27D307602D27DD26830
:1013A800D269753300120DFD120E221208D51208EB
:1013B800DC1208D51208DC1208D50213D2C2AF120B
:1013C8000F15D2AF75730075BB0E120B6012068530
:1013D800120C7B120CC51208DC120B4F306D031275
:1013E80006862067031207D830670312081F120CFD
:1013F8007B120CEA1208DC120B60306D031206C275
:10140800120C7B120D611208DC120B4F306D0312A7
:101418000720120C7B120D861208DC120B60306D4F
:101428000312077D120C7B120DFD1208DC1208391D
:10143800120B4F120C7B120E2212083D1208DC30E0
:101448006932206B2F85676485676585636C756D68
:101458000179187A0CC3E53399400CC269D26A8ABB
:0E146800357564FF02147CC3E55F94014003F8
:101476000213D20214F9306A1B206B18E53514707A
:1014860004C26A61C5F535C3E55F940140030213E2
:10149600D20214F9753600C3E5627882985054304A
:1014A6007404E52A604D7888E6B40317207D05208C
:1014B600760781C930760281C9206B07D26B8567B2
:1014C60064811178F0306B058567647820C3E54147
:1014D60098500261D2306B1BC26BC27D307602D24D
:1014E6007DD26A75351285676461D20536E55F601F
:1014F6000281FC753600C2AF120E977887E6FE763B
:1015060002120F157887EEF6E4F522F523F524F599
:1015160025F526F568C268D2AF12057C120E973003
:101526007409C3E53694054002019341A5901A0D4E
:1015360078201215B7E520B45A0CA31215B7E5208A
:10154600B4A503021555120EAC121575021574904A
:101556001A0378807B0A1215B7A308DBF9901A0FD5
:10156600788C7B181215B7A308DBF9901A2722C2CC
:10157600AF1215F61215D0901A00740E1215BCA3F0
:1015860074041215BCA374141215BC901A03788047
:101596007B0A1215BBA308DBF9901A0F788C7B180F
:1015A6001215BBA308DBF91216091215E7901A27C4
:1015B60022E493F622E6438F01538FFD75EF027501
:1015C600B7A575B7F1F0538FFE22438F02438F0103
:1015D60075EF0275B7A575B7F1901A0DF0538FFC2C
:1015E60022901A0D745AB1BC901A0E74A5B1BC2281
:1015F6007A3079D07820901A40B1B7E520F709A360
:10160600DAF7227A3079D0901A40E7B1BC09A3DA2A
:10161600F922AB77A878BB01027984BB02027985EF
:10162600BB03027986BB04027992BB05027987BBAC
:10163600060279A3BB0702799CBB08027988BB091D
:10164600027989E8F7227C05120595DCFB22C2AFF8
:101656001205A51205AC1205B31205BA12058612BB
:1016660005A51205AC1205B31205BA1205861205B8
:10167600A51205AC1205B31205BAD2AF22C2AF123B
:1016860005BA1205B31205AC1205A5120586120598
:10169600BA1205B31205AC1205A51205861205BAD3
:1016A6001205B31205AC1205A5D2AF22AE77AF78FC
:1016B600C2AF1205A51205A51205A5120586DEF212
:1016C6001205BA120586DFF8D2AF22D154D14CD119
:1016D6004C757701757801757900D1B27C05AD5FDF
:1016E600120595C3ED955F70F5C3E55F9401400A59
:1016F600C3E55F94FF403202170DD118B175D1547E
:10170600C2AF75EF12D14CDCD50579C3E5799403E8
:10171600500280C6D14C0578E5771490009F93F867
:1017260008C3E57898500280AED14CD14C0577C3FA
:10173600E577940A5002809C120EACB175C2AF7563
:04174600EF12D14C81
:0319FD00020FF5E1
:101A00000E0414FFFFFFFF03040A0101015AA501A0
:101A1000FFFFFFFFFF03FFFFFF25D0FAFA04FF01DE
:081A2000007AFF01010003FF41
:101A40002348694D6F64656C436F6F6C323241237C
:101A500023424C48454C4923463333302320202031
:101A60002020202020202020202020202020202076
:101C0000C2AFC2D353D9BF7581C043B20343FF8073
:101C1000752438752503B1C975EF0275E24043F1AB
:101C20001053A4EF75D400D2847DFA780379E67C52
:101C300010752200752300901DD67B0675249875BB
:101C400025013084028142208408D8FBD9F9DCF7D1
:101C500081B4308408D8FBD9F9DCF781B4B189E4C8
:101C600093A3C39A6004DDC381B4DBDBB17B600264
:101C7000812B7B08E493FAA3B15CDBF87A30B15C8A
:101C8000752200752300B17BEAFCEBFDC3ED94FEE9
:101C9000400EB17B8A278B28ED30E0048A828B834B
:101CA000B17B7AC270D8C3ED94FE601350CEBD00F4
:101CB00025EC60097520007521FF0200008100A855
:101CC00027A9280809D804D90281D3B17FEA89AAB3
:101CD000F281C50D81A0C3ED94035049EDA2E092BD
:101CE000007AC5C3E5829400E583941C50902000DF
:101CF00010438F02438F0175B7A575B7F1F030001F
:101D00001FA827A9280809438F01538FFDD804D99C
:101D100002A12089AAE275B7A575B7F1F0A3A10DBC
:101D2000538FFC817C7AC1BD030CE493A3FAB140CC
:101D3000DCF8B138817C817EAA22AB23B15CEBFA5E
:101D4000EA6222752608C3E52313F523E52213F57D
:101D50002250066323A0632201D526EAB1C9B1C986
:101D600075260AEAF4200102D284300102C284B14D
:101D7000C9C3134002C201D526EB22B17FEAFB2082
:101D80008402A17F308402A184752608AE24AF2589
:101D9000C3EF13FFEE13FEB1CDB1C9C3EA13308414
:101DA000024480FA30E703632201C3E52313F523DD
:101DB000E52213F52250066323A0632201D526D91C
:101DC000E52265236523F52222AE24AF250E0FDE22
:101DD000FEDFFCD20122424C48656C693437316326
:041DE000F3300601D5
:00000001FF
